:020000040000FA
:10000000B0220020150200001D0200001F020000A7
:100010002102000023020000250200000000000071
:1000200000000000000000000000000027020000A7
:1000300029020000000000002B0200002D02000039
:100040002F0200002F020000590500002F020000BF
:100050002F0200002F0200002F0200002F020000DC
:100060002F0200002F0200002F0200002F020000CC
:100070002F0200002F0200002F0200002F020000BC
:100080002F0200002F0200002F0200002F020000AC
:100090002F0200002F0200002F0200002F0200009C
:1000A0002F0200002F0200002F0200002F0200008C
:1000B0002F0200002F0200000000000000000000DE
:1000C0002F0200002F0200002F0200002F0200006C
:1000D0002F0200002F0200002F020000000000008D
:1000E0000000000000000000000000000000000010
:1000F0000000000000000000000000000000000000
:1001000000000000000000000000000000000000EF
:1001100000000000000000000000000000000000DF
:1001200000000000000000000000000000000000CF
:1001300000000000000000000000000000000000BF
:1001400000000000000000000000000000000000AF
:10015000000000000000000000000000000000009F
:10016000000000000000000000000000000000008F
:10017000000000000000000000000000000000007F
:10018000000000000000000000000000000000006F
:10019000000000000000000000000000000000005F
:1001A000000000000000000000000000000000004F
:1001B000000000000000000000000000000000003F
:1001C000000000000000000000000000000000002F
:1001D000000000000000000000000000000000001F
:1001E000000000000000000000000000000000000F
:1001F00000000000000000000000000000000000FF
:10020000DFF80CD000F02AF800480047E9090000A8
:10021000B02200200648804706480047FEE7FEE778
:10022000FEE7FEE7FEE7FEE7FEE7FEE7FEE7FEE7A6
:10023000810200000102000040EA01039B0703D095
:1002400009E008C9121F08C0042AFAD203E011F815
:10025000013B00F8013B521EF9D27047064C074D96
:1002600006E0E06840F0010394E807009847103486
:10027000AC42F6D3FFF7C8FFF415000014160000D7
:10028000F0B5A449A4484FF080540B68D4F830214D
:100290000078D4F83411551CC0F3031006D09446EE
:1002A00001270026BCF1060F03D00AE003F0FF0C83
:1002B000F6E7B4F82453DFF864C2C5F30425CCF89C
:1002C0000050DDB2062D06D1032804D1DFF854C258
:1002D000934DCCF87450551C04D09446BCF1060FD5
:1002E00003D00AE003F0FF0CF8E7D4F84452DFF83B
:1002F00038C2C5F34235CCF80050DDB2062D08D126
:10030000032806D1894DD5F800C02CF0807CC5F8B3
:1003100000C0551C04D09446BCF1060F03D00BE07E
:1003200003F0FF0CF8E74FF08045C5F80C61C5F805
:1003300010617D4D2D1F2E60DDB2062D08D10328E2
:1003400006D1DFF8E4C103250CF1640CCCF80050B1
:10035000DDB2062D10D103280ED1DFF8D4C105255A
:10036000CCF80050724D78352F60714D08352E60F5
:100370000CF104063F253560551C04D016460D4689
:10038000062E03D05BE0DEB20546F9E7ED1E012D37
:1003900055D9684D2D68684E3560664D2D1D2D6808
:1003A000361D3560634D08352D68361D3560614D4D
:1003B0000C352D68361D35605E4D10352D68361DA7
:1003C00035605C4D14352D68361D3560594D183536
:1003D0002D68594E20363560564D1C352D68361D1A
:1003E0003560544D20352D68361D3560514D24350E
:1003F0002D68361D35604F4D28352D68361D35600A
:100400004C4D2C352D68361D35604A4D30352D68E4
:10041000494E40363560474D34352D68361D3560C0
:10042000444D38352D68361D3560424D3C352D68BC
:10043000361D35603F4D40352D68361D3560551CE5
:1004400003D01646062E02D007E0DEB2FAE7D4F853
:1004500058523A4E05F04F053560551C03D01346EF
:10046000062B02D008E0DBB2FAE735480368DB0769
:1004700002D06FF001030360062A07D1C91E0229CA
:1004800004D93048016841F480610160274874381C
:10049000016841F470010160BFF34F8FBFF36F8FAC
:1004A000D4E94C104FF01022062907D1C01E0328B2
:1004B00004D9D2F808021C491C310860D2F80002A5
:1004C000002803DBD2F8040200281FDA012000F024
:1004D00041FE1521C2F800121B480368002BFCD016
:1004E000C2F8041201680029FCD0002000F032FE9E
:1004F000BFF34F8F0D48F0380168144A01F4E061F2
:1005000011430160BFF34F8F00BFFDE71149104851
:100510000860F0BDE00F00F0E80F00F0403501404A
:100520000DF0ADBA00C007403C050040FCED00E016
:10053000105600400404001020C50040E40E0040A6
:10054000000400403C17004000E401400400FA05AC
:100550000090D003380000200148006800470000E8
:100560000C000020014A024900F013B851090000B4
:100570003400002002E008C8121F08C1002AFAD186
:1005800070477047002001E001C1121F002AFBD113
:1005900070472DE9F04116460F460446002503E05A
:1005A0003946B047641C6D1C20780028F8D12846D5
:1005B000BDE8F08172B609480068C00700D000BEEF
:1005C000BFF34F8F0548E4380168054A01F4E06144
:1005D00011430160BFF34F8F00BFFDE7F0ED00E076
:1005E0000400FA050EB500210091CDE901106A461C
:1005F00044F20100FFF7DEFF0EBD10B58268C3684C
:10060000934203D000F091F9002010BD052010BDE9
:1006100029B112B1531E134203D0092070470E2096
:1006200070470160838000218160C1600846704787
:1006300010B58268C3689A1A83889A4203D800F07A
:100640007EF9002010BD042010BD000070B50A4ED8
:1006500001460A48B578FFF7D0FF04464DB10020A7
:10066000B070711C0122C81D00F040FA08B1FFF7FC
:10067000B9FF204670BD0000140000208C0200204D
:10068000F0B5244E89B01F460D00044672603FD07D
:10069000A888296882B22048FFF7BAFF002835D120
:1006A000A889A96882B21C481030FFF7B1FF002862
:1006B0002CD1202219496846FFF7BEFD60690690DB
:1006C000207C00B101208DF814008DF81C70607C36
:1006D00000B10E208DF81500E0680290A06803902C
:1006E00020680190606800900A480D4A6946083009
:1006F00000F0C8F9002809D1B0702068401C05D06E
:1007000004490122491CC81D00F0F0F909B0F0BDF0
:100710000720FBE7140000208C020020D415000005
:100720006912000010B501461048FFF781FF040070
:1007300019D10F480F4A0178515C19B1001D00F022
:10074000FBFC02E00C3000F0D1FB60B9084907481F
:100750000839FFF752FF30B905490122083904482A
:1007600000F0D4F90446204610BD00009C02002091
:100770001C0000200000002000F002B800F008B8C3
:1007800072B602480168491C0160704730000020C1
:1007900003490868401E086000D162B67047000037
:1007A000300000202DE9F041064608680C46411C47
:1007B0004FF0A0474FF0010506D005FA00F1C7F849
:1007C0000815206800F0FAF96068411C02D0002189
:1007D00000F0E2F93168A069C1F82405607D227D4E
:1007E00031681043C1F86C05D4E900123068C0F8D4
:1007F0001425C0F80C15207D012815D1A068411CD6
:1008000002D0002100F0C8F9E068411C05D0854005
:10081000C7F80855E06800F0D1F9D4E90212306851
:10082000C0F80825C0F81015BDE8F0812DE9F041A9
:10083000064608680C46411C4FF0A0474FF00105E2
:1008400006D005FA00F1C7F80815206800F0C0F9D5
:100850006068411C02D0002100F0A7F93168A0694E
:10086000C1F82405607D217D32680843C2F86C051B
:10087000D4E900123068C0F80C15C0F81425207DAA
:10088000012815D1A068411C02D0002100F08DF98B
:10089000E068411C05D08540C7F80855E06800F0C5
:1008A00097F9D4E902123068C0F80825C0F810158D
:1008B000BDE8F0812DE9FC410646C0074FF0000578
:1008C0000ED0104F00240122385D00950023114600
:1008D000019500F02BF9641C042CF4D300F01CF8F3
:1008E000B0070DD5074E0024361D0022305D0323CE
:1008F00000951146019500F019F9641C042CF4D3FD
:10090000BDE8FC81C41500000249085C012100F02B
:1009100069B90000C415000010B500242046FFF797
:10092000F3FF641C042CF9D310BD826883881A403D
:1009300003689A5C0A708168491C81607047C268CC
:1009400083881A4003689954C168491CC160704784
:1009500010B50446C0B2FFF7E5FE204610BD00000A
:1009600070B50D46044600684FF4887100F05BF9DD
:100970004FF49071206800F056F94FF4927120689E
:1009800000F051F94FF4A271206800F04CF94FF4D7
:10099000AC71206800F047F920681249C0F80413D0
:1009A0002068690740F30730090E002804DB00F1D6
:1009B000E02080F8001405E000F00F0000F1E020D6
:1009C00080F8141D206840F30730002809DB00F090
:1009D0001F02012191404009800000F1E020C0F891
:1009E000001170BD100342008AB00120FFF762FFC2
:1009F000182216496846FFF71FFC1548069015494E
:100A00004FF48070CDE9070109900723124A06A927
:100A10006846FFF735FE08B1FFF7E4FD0FA0FFF7CA
:100A2000A1FD06A8FFF712FE0028FAD19DF81800D4
:100A3000FFF778FE0028F9D19DF81800712801D041
:100A40005128EED10CA0FFF78DFDFEE7AC1500009C
:100A50003C0000203C010020571200000D0A5541C7
:100A60005254206578616D706C6520737461727486
:100A700065642E0D0A000000200D0A457869742176
:100A80000D0A0000F0B505460478154889B01646F1
:100A900040F82420124A0869121DA2F1080742F802
:100AA0002400487F385520226846FFF7C5FB049490
:100AB0002878385C48B10EB10A4A00E00022694645
:100AC000281D00F02BFA09B0F0BD0EB1064A00E077
:100AD0000022694605F10C0000F0D4F8F3E70000AD
:100AE00004000020691400000D13000030B40378E6
:100AF000054CE35C1BB130BC001D00F045BA30BCB6
:100B00000C3000F029B900000000002030B4037858
:100B1000054CE35C1BB130BC001D00F0B7BA30BC23
:100B20000C3000F08FB900000000002070B541EAE1
:100B30004201DDE904564FF0A04441EA830141EA55
:100B4000052104EB800041EA0641C0F8001770BDA2
:100B500070B541EA4201DDE904564FF0A04441EA94
:100B6000830141EA052104EB800041EA0641C0F817
:100B7000001770BD70B541EA4201DDE904564FF03F
:100B8000A04441EA830141EA052104EB800041EAE7
:100B90000641C0F8001770BD1CB500220B4600923C
:100BA00011460192FFF7D4FF1CBD1CB500220B4675
:100BB000009211460192FFF7DDFF1CBD1CB500211C
:100BC00000910B46012201911146FFF7C1FF1CBDA8
:100BD0001CB5002100910B46012201911146FFF73F
:100BE000C9FF1CBD01224FF0A043824011B1C3F8E0
:100BF00008257047C3F80C2570474058002800D0DE
:100C00000120704708B5002242504058009008BDAE
:100C1000D0F80403084000D0012070474058002855
:100C200000D00120704708B5002242504058009083
:100C300008BD0121B1EB507F01D101207047002098
:100C4000704770B50D4600F091FA04000FD00020F7
:100C5000FFF792FD207920B10020FFF78FFD1120D2
:100C600070BD0120256020710020FFF787FD002066
:100C700070BD00000149024800F060BB3C0200204A
:100C8000002000402DE9F0410546007916460F4648
:100C900000EB40012D4A01EBC00102EB810494F806
:100CA0002A1011B10820BDE8F081294951F820101F
:100CB0002868FFF7C6FF08B11120F4E73946284637
:100CC000FFF770FD66603869206030004FF0010664
:100CD0002FD03F7F4FF48E712868FFF793FF4FF4BA
:100CE000A2712868FFF78EFF28681A49C0F804131C
:100CF00028684FEA471140F30730002804DB00F171
:100D0000E02080F8001405E000F00F0000F1E02082
:100D100080F8141D286840F30730002809DB00F034
:100D20001F0106FA01F14009800000F1E020C0F83F
:100D3000001128680421C0F800150020A061E061BE
:100D400084F8290044F8140FA675ACE73C02002093
:100D5000CC150000800002002DE9F05F0546007907
:100D60004FF4017600EB400303EBC000344B03EB80
:100D700080040020636813B12B68C3F80863A3697B
:100D80004FF000096BB1E06938B1606810B12868B4
:100D9000C0F804631120BDE8F09FE26101202161E9
:100DA00005E0C4F82490A261E160C4F81C9094F8B6
:100DB0002910014302D1284600F013FA6068002888
:100DC000286803D0C0F804630020E4E74FF4A2765B
:100DD0003146FFF717FFB2464FF4927B5946286819
:100DE000FFF70BFF06464FF484712868FFF705FFF5
:100DF000804651462868FFF700FF074648EA07008B
:100E00003043EBD056EA070007D12146286800F0AE
:100E1000B9F9A169606A8142E0D8C4F818900EB1AE
:100E20000320B8E70FB10F20B5E794F8291001208F
:100E30000029296801D00860C6E74860C4E70000BF
:100E40003C0200202DE9F05F054600790B4600EBDF
:100E5000400101EBC000244901EB8004284600F06A
:100E600045F810B11120BDE8F09F62614FF0000914
:100E7000C4F82090A36084F828904FF48E784E46F2
:100E800041462868FFF7BEFE28684FF0010AC0F807
:100E900008A02146286800F0B4F9606808BBD5F8BE
:100EA00000B067690FE000BF94F8280008B10F2672
:100EB00015E041465846FFF7A0FE0028F4D0214631
:100EC000584600F09EF9206AB842F2D35746414690
:100ED0002868FFF792FE0028F9D02868C760C4F898
:100EE00014903046BFE700003C020020007900EB80
:100EF000400101EBC000044901EB8000406900287B
:100F000000D00120704700003C0200200149024847
:100F100000F0C2BA68020020002000402DE9F04134
:100F20000546164600790F46154A00EBC00102EB54
:100F3000810494F8201011B10820BDE8F081114916
:100F400051F820102868FFF77CFE08B11120F4E763
:100F500039462846FFF76AFC6660386920601EB192
:100F6000397F2846FFF7FCFC28680821C0F80015E7
:100F70000020A061E0616061012184F82010DCE7BD
:100F800068020020D01500002DE9F05F04460079CA
:100F90000E4600EBC001DFF8F0A017460AEB810512
:100FA0003046FFF746FEB0B168684FF000084FF4D6
:100FB000047910B12168C1F80893A8694FF0000BBB
:100FC00080B1E86948B1686810B12068C0F804933E
:100FD0001120BDE8F09F1020FBE7EF614FF0010802
:100FE0002E6102E0EE60C5E9067B00254FF48871B2
:100FF0002068FFF718FE4FF4A2712068FFF713FE78
:101000002068C0F83465C0F838752068B8F1000F62
:1010100012D0D0F8001241F02001C0F8001220795F
:10102000D04600EBC0010AEB8100406838B120686F
:10103000C0F804932846CCE701210160EFE74FF4A4
:10104000887A4FF4A27951462068FFF7E7FD0746FA
:1010500049462068FFF7E2FD06464FF4927120688A
:10106000FFF7DCFD014647EA06000843EBD0227992
:1010700002EBC20308EB8302C2F818B001B10325EA
:10108000002ED7D00F25D5E7680200202DE9F047C4
:1010900004460E460079274900EBC00001EB8005AD
:1010A00017463046FFF7C5FD30B1204600F044F842
:1010B00020B11120BDE8F0871020FBE76F61AE6022
:1010C0004FF490774FF0000839462068FFF7ABFDEA
:1010D0004FF4AC7631462068FFF7A5FD2068AA687A
:1010E0006969C0F84425C0F8481520684FF0010927
:1010F000C0F808906868D0B9BA4651462068FFF732
:101100008DFD074631462068FFF788FD0743F4D080
:1011100010B14FF00F0808E02068C0F80C9031467D
:101120002068FFF77BFD0028F9D000206861404669
:10113000C0E70000680200200079054900EBC0000C
:1011400001EB80004069002800D0012070470000BA
:101150006802002003490860034801680029FCD0A8
:101160007047000004E5014000E401400349884263
:1011700001D1034870470020704700000020004064
:101180000C00002070B5054688690C4600284FF415
:10119000847128460AD0FFF735FDD5F81805626A34
:1011A000E1688854606A401C606270BDFFF72AFDE8
:1011B000D5F8180570BD1FB501238DF80030CDE9B5
:1011C0000121D0E90012684690471FBD1FB50123D9
:1011D0008DF80030CDE90121D0E900126846904732
:1011E0001FBD10B5044600684FF49271FFF70AFD69
:1011F0004FF484712068FFF705FD2068012101602C
:1012000010BD70B50C4605464FF48E71FFF7FAFC21
:10121000216AA068415C206A401C2062C5F81C1548
:1012200070BD1FB500228DF80020029181680191E8
:101230004261D0E90012684690471FBD1FB50022E9
:101240008DF800200291816801914261D0E900127D
:10125000684690471FBD0178022901D0012902D1BB
:101260004068FFF7BFB970477CB50178254DA1B341
:1012700001290BD002291DD18DF80010C068691C0E
:1012800001900122C81DFFF731FC30E0017A59B10D
:10129000406801781C48FFF7CBF91B4C012650B180
:1012A0008DF8006001900DE016490122491CC81D0F
:1012B000FFF71CFC7CBDA068E168814205D00020DE
:1012C0008DF80000696868468847A068E168081AD8
:1012D000A1888842E8D9AE707CBDFFE70A48094979
:1012E0001030FFF78AF930B103208DF800006968EB
:1012F00068468847F0E70349012201F10800FFF73B
:1013000005FCE9E7140000208C0200201FB50A4606
:1013100001788DF8001041680191017A8DF808106C
:10132000C0680390044850F82210001F50F8222093
:10133000684690471FBD0000080000202DE9FF47C8
:101340000C4605464FF40071FFF762FC01274FF48D
:101350000178002618B34FF4927949462846FFF7E2
:101360004CFCE0B149462846FFF74CFCC5F8088321
:1013700094F8290000B96F6002208DF80000D5F8BC
:101380008004C5F880040390A0690290E068019091
:10139000A661E661D4E900126846904728E004217E
:1013A0002846FFF735FC18B34FF484712846FFF741
:1013B00024FCE8B121462846FFF7E4FE616AA069F3
:1013C000884215D1E06938B1E268616AA06120699C
:1013D000E6616662E06008E094F8290000B96F6099
:1013E000C5F80883A661E268616A2046FFF7E3FE5C
:1013F0004FF48E7841462846FFF7FFFB80B16069C5
:10140000216A814202D294F8280028B34146284636
:10141000FFF7F8FB606918B161692046FFF701FF2B
:101420004FF4A27841462846FFF7E7FB002818D082
:1014300041462846FFF7E6FB94F8290000B12F60EB
:10144000A06900280DD0A661E268616A04B0204658
:10145000BDE8F047FFF7AFBE21462846FFF7D1FEB3
:10146000DEE7BDE8FF8700001FB50A4601788DF86A
:10147000001041680191017A8DF80810C06803904E
:10148000044850F82210001F50F822206846904768
:101490001FBD0000080000202DE9FF410C464FF45D
:1014A000927705463946FFF7B9FB0026B8B13946B1
:1014B0002846FFF7B8FB02208DF80000D5F880041D
:1014C000C5F880040390D5F83C050290E0680190CF
:1014D000A661E661D4E900126846904723E04FF424
:1014E000887739462846FFF799FBE0B13946284608
:1014F000FFF799FBD5F83C15A069884213D1E06944
:1015000060B1E268D5F8000220F02000C5F80002C2
:10151000E069A0612069E661E06001E0A661E2683F
:101520002046FFF753FE4FF4A27739462846FFF7CF
:1015300075FB68B139462846FFF775FBA06938B1DD
:10154000A661E661D5F83C152046E268FFF73EFE4D
:101550004FF4907631462846FFF760FB60B1314684
:101560002846FFF760FB0120E860606920B1D5F8EC
:101570004C152046FFF762FE4FF4AC763146284604
:10158000FFF74CFB00280ED031462846FFF74BFBF7
:101590006069002807D0D5F84C1504B02046BDE896
:1015A000F041FFF74BBEBDE8FF81000008000000DE
:1015B0000600000005000000070000000000000019
:1015C00000E0D701111213140D0E0F10750C00005E
:1015D0000D0F0000FFFFFFFFFFFFFFFFFFFFFFFFFB
:1015E000FFFFFFFF00000000000000000000D60128
:1015F0000601000014160000000000203C0000005E
:1016000074050000501600003C0000207422000009
:101610008405000000000000000000000000000041
:1016200000000000000000000000000000000000BA
:1016300000000000002000400000000000200040EA
:101640000000000000000000000000000090D00337
:0400000500000201F4
:00000001FF
